:040000007AC5FECFF0
:10000400FDCFFCCFFBCFFACFF9CFF8CFF7CFF6CFA8
:10001400F5CFF4CFF3CFF2CFF1CFF0CFEFCFEECFD8
:10002400EDCFCDC0C6CCC8203E3E3E3E3E3E202055
:1000340000002A20526144694B614C32202A20007E
:10004400C0C2D2CECFCEC8D1CA20202020200000EA
:10005400C02ECFCEC8D1CA203E3E3E3E3E20000038
:10006400D02ECFCEC8D1CA20202020202000D02ED0
:10007400CFCEC8D1CA203C20203E20200000CFCEC5
:10008400C8D1CA20C2C2C5D0D52020200000CFCEFE
:10009400C8D1CA20C2CDC8C7202020200000CDC0AE
:1000A400D1D2D0CEC9CAC0202020202000000C010B
:1000B4000B0A04140A01320A05151E04281E012025
:1000C4001E050A28041E28012928050A29042A29AC
:1000D400012829052B32042832050A0000000B00F0
:1000E40000A8060A36000000140000F906150000F6
:1000F40006071E4400000020540015072864000071
:100104000029720000002A820052072B92006F0718
:1001140032A200000000000000001027E803640081
:100124000A0001000010000110000100000000009E
:100134000000005F00000007000700147F147F1414
:10014400242A7F2A12231308646236495522500058
:1001540005030000001C2241000041221C00140879
:100164003E081408083E080800503000000808083B
:10017400080800606000002010080402000000006D
:100184000000005F00000007000700147F147F14C4
:10019400242A7F2A12231308646236495522500008
:1001A40005030000001C2241000041221C00140829
:1001B4003E081408083E08080050300000080808EB
:1001C400080800606000002010080402000000001D
:1001D4000000005F00000007000700147F147F1474
:1001E400242A7F2A120684FE8406364955225000AA
:1001F40005030000001C224100007F3E1C08140877
:100204003E081408083E080800503000000808089A
:100214000808006060000020100804023E514945AF
:100224003E00427F400042615149462141454B31E5
:100234001814127F1027454545393C4A4949300175
:10024400710905033649494936064949291E0036CC
:10025400360000005636000008142241001414141D
:10026400141400412214080201510906324979414B
:100274003E7E1111117E7F494949363E414141225A
:100284007F4141221C7F494949417F090909013EB7
:100294004149497A7F0808087F00417F4100204096
:1002A400413F017F081422417F404040407F020CBF
:1002B400027F7F0408107F3E4141413E7F090909C6
:1002C400063E4151215E7F09192946464949493173
:1002D40001017F01013F4040403F1F2040201F3F5C
:1002E4004038403F631408146307087008076151DD
:1002F400494543007F414100020408102000414168
:100304007F00040201020440404040400001020416
:100314000020545454787F4844443838444444209A
:10032400384444487F3854545418087E0901020C58
:100334005252523E7F0804047800447D400020401D
:10034400443D007F1028440000417F40007C041895
:1003540004787C0804047838444444387C14141425
:1003640008081414187C7C080404084854545420C5
:10037400043F4440203C4040207C1C2040201C3C46
:100384004030403C44281028440C5050503C4464B5
:10039400544C44000836410000007F000000413600
:1003A400080010080810087846414678000000004C
:1003B4000000005F00000007000700147F147F1492
:1003C400242A7F2A122313086462364955225000D6
:1003D40005030000001C2241000041221C001408F7
:1003E4003E081408083E08080050300000080808B9
:1003F40008080060600000201008040200000000EB
:100404000000005F00000007000700147F147F1441
:10041400242A7F2A12231308646236495522500085
:1004240005030000001C2241000041221C001408A6
:100434003E081408083E0808005030000008080868
:10044400080800606000002010080402000000009A
:100454000000005F00000007000700147F147F14F1
:10046400242A7F2A12231308646236495522500035
:1004740005030000001C2241000041221C00140856
:100484003E081408083E0808005030000008080818
:100494000808006060000020100804023E5149452D
:1004A4003E00427F400042615149462141454B3163
:1004B4001814127F1027454545393C4A49493001F3
:1004C400710905033649494936064949291E00364A
:1004D400360000005636000008142241001414149B
:1004E4001414004122140802015109067E1111114D
:1004F4007E7F494949317F494949367F01010103DA
:10050400702927217F7F4949494177087F0877412E
:10051400414149767F1008047F7F1009047F7F08DA
:1005240014224120413F017F7F020C027F7F080893
:10053400087F3E4141413E7F0101017F7F09090956
:10054400063E4141412201017F010147281008076D
:100554001E217F211E63140814633F2020205F079F
:100564000808087F7F407F407F3F203F205F017F56
:100574004848307F4830007F007F4848304141413F
:10058400493E7F083E413E462919097F2054545470
:10059400783C4A4A49317C545428007C0404040CB5
:1005A400722A26227E38545454186C107C106C44E1
:1005B400445454387C2010087C7C2112097C7C1023
:1005C40028440020443C047C7C0810087C7C1010E7
:1005D400107C38444444387C0404047C7C14141493
:1005E40008384444442004047C04044428100804C7
:1005F40008147E140844281028443C40407C400CD5
:100604001010107C7C407C407C3C203C207C047C92
:100614005050207C5020007C007C505020284444C2
:1006240054387C10384438485434147C0080C0E07A
:10063400E060E0E0C08000000000000070FFFF0107
:1006440000000000FFFFFE0000000000000F1F3C40
:10065400383038381F0F030000000000000000008D
:1006640080E0E00000000000000000000000030340
:1006740003FFFF0000000000000000000000383805
:10068400383F3F38383800000000000000C0C0E0A8
:100694006060E0E0C0800000000000000001000095
:1006A40080C0E0F93F1F000000000000003C3E3F16
:1006B4003F3B3938383838000000000000C0E0E023
:1006C4006060E0E0C0C00000000000000001000025
:1006D4003030387DEFCF000000000000001C3838B7
:1006E4003030383C1F0F0100000000000000000003
:1006F4000080C0E0E000000000000000E0F0F8DE50
:10070400CFC7C1FFFFC0C000000000000000000010
:100714000000003F3F0000000000000000E0E0E0B7
:10072400E0E0E0E0E0E0E00000000000003F3F3FE8
:1007340038383070F0E0000000000000001C383849
:100744003030383C1F0F030000000000000080C060
:10075400C0E06060E0E0000000000000E0FEFF3761
:1007640039181838F0F0C00000000000000F1F1CFA
:10077400383030381F0F07000000000000E0E0E0D0
:10078400E0E0E0E0E0E0E000000000000000000045
:1007940080E0F87E1F070100000000000000383EE2
:1007A4001F07010000000000000000000080C0E0FE
:1007B400E06060E0C0C000000000000000CFFF7FE8
:1007C40038307070FFEFC70000000000030F1F3CBB
:1007D400383030381F1F0F00000000000080C0E0D8
:1007E400E060E0E0C0800000000000000C3F7FF10A
:1007F400E0C0C0E1FFFFFE00000000000000383050
:100804003038381E0F070000000000000000000010
:1008140000000000000000000000000000000000D4
:100824000000000000000000000000003C3C3C0010
:1008340000000000000000000000000000000000B4
:100844000000000000000000000000000000404024
:10085400404040FEFE404040404000000000000098
:100864000000000F0F000100000000010000000064
:100874002920202000293E202000293E3E20002956
:100884003E3E3E00D1D2C5D0C5CE00CCCECDCE208A
:10089400200025303275002A20526144694B614C96
:1008A40032202A000080C0E0E060E0E0C080000068
:1008B4000000000070FFFF0100000000FFFFFE00C9
:1008C40000000000000F1F3C383038381F0F0300B1
:1008D400000000000000000080E0E00000000000D4
:1008E400000000000000030303FFFF0000000000FD
:1008F4000000000000003838383F3F383838000026
:100904000000000000C0C0E06060E0E0C0800000C3
:10091400000000000001000080C0E0F93F1F00005B
:1009240000000000003C3E3F3F3B39383838380077
:100934000000000000C0E0E06060E0E0C0C0000033
:1009440000000000000100003030387DEFCF0000CF
:1009540000000000001C38383030383C1F0F010004
:1009640000000000000000000080C0E0E000000083
:1009740000000000E0F0F8DECFC7C1FFFFC0C000F8
:1009840000000000000000000000003F3F000000E5
:100994000000000000E0E0E0E0E0E0E0E0E0E00093
:1009A40000000000003F3F3F38383070F0E00000A6
:1009B40000000000001C38383030383C1F0F0300A2
:1009C40000000000000080C0C0E06060E0E00000C3
:1009D40000000000E0FEFF3739181838F0F0C000BE
:1009E40000000000000F1F1C383030381F0F0700B4
:1009F4000000000000E0E0E0E0E0E0E0E0E0E00033
:100A0400000000000000000080E0F87E1F070100E5
:100A1400000000000000383E1F0701000000000035
:100A2400000000000080C0E0E06060E0C0C00000A2
:100A34000000000000CFFF7F38307070FFEFC70068
:100A440000000000030F1F3C383030381F1F0F0018
:100A5400000000000080C0E0E060E0E0C080000032
:100A6400000000000C3F7FF1E0C0C0E1FFFFFE008A
:100A740000000000000038303038381E0F07000036
:100A84000000000000000000000000000000000062
:100A94000000000000000000000000000000000052
:100AA400000000003C3C3C0000000000000000008E
:100AB4000000000000000000000000000000000032
:100AC4000000000000004040404040FEFE40404026
:100AD40040400000000000000000000F0F00010073
:100AE40075016A08080006006C0839027801A80834
:100AF4000000F894EE27ECBBF1E0FBBFEBBFE5BFD1
:100B0400F8E1F1BDE1BD8DE0A2E0BB27ED938A954C
:100B1400E9F780E094E0A0E6ED930197E9F7E2EECF
:100B2400FAE085919591009761F0A591B5910590B2
:100B34001590BF01F00105900D920197E1F7FB01BB
:100B4400F0CFEFE5EDBFE4E0EEBFC0E6D1E002C2D6
:100B5400AAD81B8100E0B2D4B7D499F0AFD40F0166
:100B6400A491EB81EA1731F4F0013196A491EA8162
:100B7400EA1709F004C0A2D43296149102C00F5FA0
:100B8400EACFE12F97D8E0C00FD6E0ECEA9340D645
:100B94009ED4EC91EA939ED4A181AA939BD4A28182
:100BA400AA9398D4A381AA9395D4A481AA9330D666
:100BB4000AD62CC4F9D5E1ECEA932AD68FD487D48B
:100BC400EC938CD4A881B9811196EC9387D4A88135
:100BD400B9811296EC9382D4A881B9811396EC93CF
:100BE4007DD4A881B9811496EC93EDD50FC479D442
:100BF400A0E0B0E043D8E0916101A1E0B0E03ED8CC
:100C0400E0916201A2E0B0E039D8E0916301A3E091
:100C1400B0E034D8E0916401A4E0B0E02FD864D40B
:100C24006CD4E92DABE1B0E029D8089570D4E091FB
:100C3400680173D4BAD71E2F113010F0143008F0A5
:100C440006C06DD46CD4A6D3E4E7F8E06BD41430BA
:100C540010F0183008F006C062D461D49BD3E9E7E1
:100C6400F8E060D4183010F01C3008F006C057D4F7
:100C740056D490D3EEE7F8E055D41C3010F0103180
:100C840008F006C04CD44BD485D3E3E8F8E04AD44A
:100C940008C03DD4E0916701EF771E2F46D448D4B5
:100CA400D0D5E12F19910895E5E6F1E041D482DF32
:100CB400E0916701E078E03831F4E0E33CD46AD3B2
:100CC400E8E8F8E005C0E0E336D464D3EFE8F8E000
:100CD400FA93EA9373D30895249706D4E0E0F0E4FA
:100CE4006CE176E4F8D6E6D55F01D501E0E1F7E200
:100CF40024D4E88327D411F4E0E202C0E881E05D63
:100D0400E883D501E8EEF3E018D4E05DE983D5018A
:100D14001CD413D4E05DEA83D50107D40ED4E05D7E
:100D2400EB83E881EA93EAE013D4E981EA93E6E10C
:100D34000FD4EA81EA93E2E20BD4EEE2EA9308D418
:100D4400EB81EA93E3E304D424960895E0917501DA
:100D5400E030B9F0E0E0E0937501ABE1B0E07AD7C0
:100D64009E2EF8D3FCD3FFD302D40DD40FD41CD4BD
:100D74002CD3D5D3E5E0EA930DD3EBE9F8E0D8D34F
:100D84003FD3EAE0DBC212D41AD407D61DD4ACD3C5
:100D9400A433EFE2BE07EEEC8E07ECE49E0729F4E1
:100DA400ECE9F4EE66EA7CE40FD417D409F03DD400
:100DB400C9D309F4CFD3D3D3C1C2F8D300D4E6D571
:100DC40003D492D3A83CE3EBBE07E6EA8E07ECE437
:100DD4009E0729F4E0E6FEEF6DEC7CE4F5D3FDD349
:100DE40009F023D4AFD309F4B5D3B9D3A7C29394EC
:100DF400EAE0E91511F4E1E09E2E1CD425D4C3D316
:100E0400C5D3D2D349D49AC2E92D87D331979E2E24
:100E1400992011F4EAE09E2E0DD416D4B4D3B6D39F
:100E2400C3D33AD48BC2E4EFFCEE6EEB7CE4CCD3B8
:100E3400EAE08E1678F583946620A1F4E1E0EA9363
:100E4400A2DFEAE3F0E02FD424DFE73330F021DF40
:100E5400EF3318F4EBDEE93008F402C0E1E06E2E63
:100E64003BDFEACF41D349D3E82D1FD4D001FED6CE
:100E74008AD3E6E9F8E05CD3E82DFF2766277727D5
:100E8400E0D684E010D22896EDE155D38DD39DD2DF
:100E94006624CECF88245ED362D310D4EAE04EC257
:100EA400662091F442D3FFD3E1E0EA936CDF09D4E6
:100EB40030F0EFDEEF3318F4B9DEE93008F402C0A5
:100EC400E1E06E2E09DFECCF0FD317D3E92DEDD37C
:100ED40000D445D3F3D3E9E231C2662091F425D39B
:100EE400E2D3E1E0EA9369DFECD330F0D2DEEF3312
:100EF40018F49CDEE83008F402C0E1E06E2EECDE6B
:100F0400ECCFF2D2FAD2E92DD0D3E3D328D3D6D37F
:100F1400E9E214C2C8D6E6E9F0E0C5D3809902C07C
:100F240011E009C0819902C015E005C0829902C090
:100F340014E001C010E0103029F0CC2019F4D12EB7
:100F4400E1E0CE2ECC2019F00D2DCC2401C000E020
:100F5400E02F1EC22197EFEFE7BBE0E8E8B91FD40A
:100F6400CDD1A0E0B0E076D6E0936001A1E0B0E09E
:100F740071D6E0936101A2E0B0E06CD6E093620127
:100F8400A3E0B0E067D6E0936301A4E0B0E062D6EA
:100F9400E09364014AD3E3D2ECE01E2F5E2EE6E236
:100FA400F0E09BD328EA36E09DD3309761F0B7D2C6
:100FB400E5E0EA93EFD196D3BBD222D2E0E0E0930E
:100FC4007601E0937701A6DF0E2F022E032A21F08B
:100FD4000A93F901099505C0003021F05A920A9349
:100FE400B7DD1E2F5116B9F0512EE0E0E8837FD310
:100FF4006BD289F07CD3A4915A1649F478D33196F4
:101004001CD66BD374D3339618D69F0104C0E881E1
:10101400EF5FE883ECCF0ADE47DEC6CFFFCF43D6CF
:101024006DD3129601D63097F1F068D36AD38F014D
:10103400309761F00230E0E01E07A0F0F80131972C
:101044008F01AA81BB811496ED93FC9357D312961A
:101054005BD33197AC81A08351D3E6D5FF2312F043
:101064004DD352D305C04AD3EFEFFFEFED93FC937A
:1010740021D625960895269712D610E0AC85BD8515
:10108400E0E0F0E0ED93FC93EA89FB893196EA8B8A
:10109400FB8B3197E4912E2FE03009F4FEC0E12F51
:1010A400E03031F4253211F411E001C033D3F4C03F
:1010B400E130A1F4253211F42DD3EDC012E040E06B
:1010C40000E02D3211F401E0E7C02B3211F44BE2C1
:1010D400E3C0203211F440E2DFC002C0E23039F450
:1010E40050E013E0203311F40068D6C003C0E330AD
:1010F40009F0D2C0203310F02A3308F007C0AAE068
:101104005A9F502DE22FE0535E0FC6C0E22FE33604
:1011140039F408D30AD306D3A481AA930AD3BBC053
:10112400E33731F40DD30ED310D3B3D11E2F08C03F
:10113400E03751F405D306D308D3B5D11E2F086088
:1011440002600F7730E02EC0E43611F0E93611F476
:10115400046002C0E53729F4EEE1F1E0F9D215E0CC
:101164000BC0E83511F4086003C0E83709F093C0F8
:10117400E8E2F1E0EDD214E002FF11C0E1D2E2D2E4
:10118400EAD2AB85AA232AF4EA85FB85EDD4E3D21F
:101194004DE2403011F01F5F01C00B7F03C0D0D27D
:1011A400D1D2D9D200FD10C0151770F407FF08C0C2
:1011B40002FF04C00B7F242F115001C020E301C0A3
:1011C40020E2A8D25150F0CF312F01FF15C03030AA
:1011D40091F003FF05C0EE81FF812591B9D205C0CE
:1011E400AE81BF812D91AE83BF8394D2503009F07C
:1011F40051503150ECCF46C020E3EE81FF811DD524
:10120400E887F987EE81FF813296A2D2E885F985D5
:10121400AA85BB85AE17BF0748F02F5FA885B9859F
:10122400EA85FB85EA1BFB0B96D2F0CF2A3328F024
:1012340003FF02C0295F01C0295D04FD19C02133E9
:1012440020F4A885B985119709F409C0531710F043
:1012540000FF01C011C020E207FF0AC020E30061C3
:1012640002FF06C00B7F4A9364D2503009F05150FC
:1012740051D2503009F051503150A885B985129798
:1012840008F0BACF00FF07C0503029F05150E0E217
:10129400EA934FD2F9CF10E0F7CEAC85BD85C4D424
:1012A40005D564960895FF92F82E2697FAD456D25F
:1012B400309719F4EFEFFFEF1DC0DE01169650D4FE
:1012C4008D014CD245D2E0E0E887E987DE011A9629
:1012D40047D4AAD42DD11A930A93E1E1F8E028D196
:1012E400FE013A9625D1C7DE9F01AE81BF81E0E0C1
:1012F400EC93F901DDD42A96FF900895C09AC09822
:1013040024D1D1D1C09AE1E22ED2E8EC2CD2E3E18F
:101314002AD2E0E228D2E9E026D22BD0E8E023D298
:10132400ECE021D2FCD0FBD035D00895C19801C0A7
:10133400C19AC498E881EA9303D0C49A2196089587
:10134400B2D408E010E00024001601067CF4C3982F
:10135400EA81E078E03811F4C29A01C0C298C39AD5
:10136400EA81EE0FEA8301501040EDCFA3D4239617
:10137400089599D4D4D0D3D00DD008EF11E000242F
:10138400001601062CF4CBD0D3DF01501040F7CF68
:1013940094D40895E881E770E064E5D1E981E068D8
:1013A400E2D134C01A9310E0153020F4DED1EAD132
:1013B4001F5FFACFB4D0BCDF188128C0E5D184D038
:1013C40019F0E5D1EFDFFACF21C081D0EC91E03004
:1013D40039F07DD0ED91A883B983EA93E3DFF5CFAB
:1013E40015C01A93EFEFCED110E0153028F4BDD11B
:1013F400E095C8D11F5FF9CFEFEFC4D1188106C0C3
:10140400C3D162D019F0C3D1ECDFFACF229608958C
:1014140048D4AD81AE3211F4EAE00CC0AD81AB32F8
:1014240011F4EBE007C0AD81A03211F4ECE002C08E
:10143400ED81EF70ED8310E01330F8F4EC81ED5F93
:10144400EA93E12FEF5FEA93A5DF00E0003198F41F
:10145400ED81A0E3EA9FF001E858FE4FDF01E12FA0
:101464005CD09AD3AE0FBF1FEE27A00FBE1FEC9126
:1014740089D10F5FEBCF1F5FDFCFAD81AE3219F49F
:10148400EC81EB5F02C0EC81E45FEC8311D426961F
:101494000895A991B991EE27FF276D91662311F064
:1014A4003196FBCF0895AA27BB27E991F9910590BE
:1014B400002011F01196FBCFFD010895A3E00A9FCF
:1014C400F001EE54FF4F0895E491E0300895A881AF
:1014D400B98108959DD1E881F9810895E1E0EA9305
:1014E4007CC1E09160010895A0916A01B0916B0103
:1014F40080916C0190916D010895E0E0F0E563EC5A
:1015040077E4E9D2A5E0B0E0D5D1B0D308951A9339
:10151400E5E6F1E0FA93EA934DCBF0E00895E0E0DC
:10152400EA930895FA93EA9349CFEAE0F0E0089544
:10153400FA93EA930895EA93F2CF60D3DF01F5DFDB
:1015440070D30895E881E0300895E4E6F0E008956A
:10155400EA935ECFC6DFEF77E09360010895E0E69B
:10156400F1E0E6DF11CBA5E0B0E070D30895662783
:101574007727A0EAB6E881E090E020D3AAE6B1E0BC
:10158400D0D156D30895E2E7F1E0D2CFE6E9F8E00E
:10159400CFDFE92DFF276627772753D384E083DE47
:1015A40028969ADBEDE1C7CFF5DEEDCFE0916A0135
:1015B400F0916B0160916C0170916D010895A0E050
:1015C400B0E583EC97E40895E0936A01F0936B012E
:1015D40060936C0170936D010895E8DFA0E0BAEBAD
:1015E4008BE598E4D3D1A0E0B0E080E890E425D284
:1015F400DF01CB01E0E0F0E060E077E46CD2AEE63E
:10160400B1E058D115D3A0916E01B0916F018091D2
:10161400700190917101E8E0B3D2EF73E09360013F
:10162400E0916E01E09361018DCF5BDFE068E093B0
:1016340060010895E92DA7E0B0E06FDFEE0FFF1F12
:10164400AE0FBF1F03D393CFB1DFA0E0BAEB8BE59E
:1016540098E49CD1A0E0B0E080E890E4EED1DF0112
:10166400CB01E0E0F0E060E077E435D2AEE6B1E053
:1016740021D1DED2A0916E01B0916F0180917001F1
:1016840090917101E8E07CD2EF73E0936001E09106
:101694006E01E093610163CF98DEA9DA56DF48DF7B
:1016A400D0D0EAE0089544DFCCC0A7E0B0E035DF55
:1016B400EE0FFF1FEA0FFB1F0F0155CF98DA45DF2E
:1016C400F2CF95DAB3DA4E2EE4DA7E2EE2DAE7339D
:1016D4000895D001CBD266243DCFE0937601F093F8
:1016E40077010895E0917601F09177010895E881FA
:1016F400A5E0EA9FF001EE51FF4F0895AA81BB8156
:101704000895149691D20895ED91FD913196FE932A
:10171400EE9308952A93ED85FE850ADFE989FA8917
:1017240009950895E889F98908953497E88BF98B28
:101734000895ED85FE85FCDEE989FA890995089509
:10174400F1DFF3CFA889B989DCCFEE83FF83F0CE34
:10175400EE83FF830895EA87FB870895DE011C96D4
:10176400FFD162D20895EA93E1CDE981A5E0EA9F31
:10177400F001E05DFE4FDF01E12FCFDEEA0FFB1F3A
:10178400E4910895EA93D4CDE881F9810895FCDFCA
:101794003196E883F9833197E491EA930895A998FF
:1017A400A898A19AA09815C0A098A198EE27000027
:1017B400989B0895999B089504D0A09A02D0A19A69
:1017C400E1E062E007C0A09AA19A03D0A198F9DFF2
:1017D400A09863E06A95F1F7089578E0A198F1DFA5
:1017E400999BFECFEEDF889498990894A19AF1DF33
:1017F400EE1F7A9599F77991772311F4A09801C097
:10180400A09ADFDFA198E5DFA19ADBDFA098D9CF0A
:10181400E99178E0EE0F10F4A09801C0A09AD9DF06
:10182400A198CFDF999BFECFCCDFA19A7A9591F74F
:10183400A098C7DFA198CDDFE1E09899EE27A19A9F
:10184400C0CFE991F991309639F08AEF90E0019791
:10185400F1F7A8953197C9F70895552342F4503804
:1018640011F4E0FF04C03196691F791F6BF050E852
:10187400572711F45F93CFC05F3F31F0660F000C20
:1018840057956795752F08955F9300200AF0CFC090
:10189400C8C050E8192E1522880F991F9527550F97
:1018A400879550E8072E0522660F771F7527550F79
:1018B40067950895689401C0E8945F93F2DF7038E7
:1018C40018F07F3F08F4A7C056E1571BAAF45195BE
:1018D40058300EF4593030F0EFEFFFEF6FEF7FE741
:1018E40077F91AC077275523B9F0EE0FFF1F661F4B
:1018F400771F5A95D1F710C07727583028F0EF2F6B
:10190400F62F672F5850F9CF552331F07695679508
:10191400F795E7955A95D1F700200AF429D15F91FC
:101924000895689401C0E894309760407040B1F025
:10193400002426F0772312F400941AD1172E7EE1A6
:10194400112032F07A95EE0FFF1F661F111CF9CF9C
:10195400EF2FF62F612D5F938ADF5F9108954F93E8
:10196400AF01FD01DA01AB01BC01CA01402D012C1C
:10197400142E4F910895EA0FFB1F681F0895E095F8
:10198400F0956095EF5FFF4F6F4F08955F9381DF90
:10199400903871F150E8152604C05F937ADF9038CF
:1019A40039F1703821F1572F591B2BF112F4D7DF7D
:1019B400FACF583118F0AA27BB278827583028F0C7
:1019C400AB2FB82F88275850F9CF552329F0869587
:1019D400B795A7955A95D9F7502D512572F0CBDFBD
:1019E40038F46795F795E795739513F420C0B7DF3E
:1019F4003EDF5F910895D8F7FBCFEA1BFB0B680B22
:101A040051F010F40094BBDF662392F3EE0FFF1F36
:101A1400661F7A95CBF7EE27FF27662777275F9116
:101A24000895EFEFFFEF6FE77FEF5F910895EFEF1A
:101A3400FFEF6FE77FE75F9108955F932ADF7038C8
:101A440051F3903841F301240894791F23F41CF3D3
:101A540000203AF3ECCF0F921F932F933F934F93B1
:101A6400112722279927689FA0018F9F302D410DB0
:101A7400591F6B9F300D411D591F8E9F27D0BF9F4B
:101A840025D06A9F23D0BE9F1DD0AF9F1BD0AE9F91
:101A9400110D291F391F491F591FE32FF42F652FDB
:101AA400522F4F913F912F911F910F9066232AF04F
:101AB400550FEE1FFF1F661F02C073954BF2CDDE5C
:101AC4005F910895100D211D391F02C0200D311D95
:101AD400491F591F08955F93DCDE703821F41120EB
:101AE4000AF49FCFA4CF903809F495CF0124089429
:101AF400970B1BF4D4F30020F3CF792F1F932F936C
:101B04003F934F9311241127222733274427552726
:101B140090E2AE17BF078607410730F0AE1BBF0B3C
:101B2400860B410B089401C08894551F221F331F54
:101B3400111CAA1FBB1F881F441F9A9551F7F90156
:101B4400612D4F913F912F911F91662332F0550FD4
:101B5400EE1FFF1F661F7A9543F27FDE5F910895A3
:101B64000024AF0DB01D0895F195E195F04008955E
:101B7400F09560957095E195FF4F6F4F7F4F0895F5
:101B8400EE230E2EFD01BC0131F076956795F79595
:101B9400E7950A94D1F70895EE0FFF1FEE0FFF1F8C
:101BA400EE0FFF1FEE0FFF1F0895F595E795F595CE
:101BB400E795F595E795F595E79508957A9F702D46
:101BC4006B9F700DF89F700DE99F700D6A9F602DDB
:101BD400710DFB9F600D711DE89F600D711D8827BD
:101BE400FA9FF02D610D781FEB9FF00D611D781F9A
:101BF400EA9FE02DF10D681F781F08950024112439
:101C040090E1AA0FBB1F001C111C0E1A1F0A18F426
:101C14000E0E1F1E01C0A1609A9599F7FD01D00117
:101C24000895ECDFFD010895ED91FC91119708955D
:101C3400ED93FD936D937C9308950590F491E02DBD
:101C440008957A936A93FA93EA930895119602D0C9
:101C5400FE2F1197E199FECFFF93FFB7F894AEBB27
:101C6400BFBBE09AEDB3FFBFFF91089507D0119673
:101C7400EF93EF2F03D0EF9111970895E19B02C0EA
:101C8400A895FCCF9FB7F894AEBBBFBBE09A8DB3C9
:101C9400E81719F0EDBBE29AE19A9FBF08955A93B1
:101CA4004A933A932A931A930A9308955D814C8137
:101CB4003B812A8119810881089509911991089518
:00000001FF
